S111FFF2F800F804F808F80CF810F814F818E1
S11BF8006E9F00026E9F00046E9F00066E9F00086E9F000A6E9F000C74
S11BF8181A504F97141F8BB72021B72023B7204CB7204BCCFFF0B720FD
S11BF8304FF72043CCFF3FB72040F7204286CEB7204C867FB7204EB741
S11BF848204D10CE00008EF8898608AFE15A26FB8EF8189F0E10CE0088
S11BF8602F860E8D78BDF93BC10D271DC60C81E62711C60A8178270B55
S11BF878C60881802705C6064D26E2CA10F720133F1A504F1F8B10DFC3
S11BF8902110CE00618D61863E8D52B620100F14BDF93BD715108EF8EF
S11BF8A8BBA6A027F3AEA1911526F68D388D7097146E8447F99D4DF996
S11BF8C0A140F9A150F9C653F9E152FA3523FA3544FA9B57FAB54CFB7C
S11BF8D8160DF89100B72011840F8A10B72013860BB7201239F620118F
S11BF8F0C51027F9B7201039860D8DF1860A20EDA68027048DE720F85C
S11BF90839A68097158D049615200444444444840F8B30813923CE8BE4
S11BF9200720CA8DE48DE2862020C28D008DF620F48DC58E00128DEBE4
S11BF9389E1239F62011C50827F9B620101F89C47FC1612D06C17A2E27
S11BF95002C0200D142708DD171F988D90DC17398DD9C030102BFF29BC
S11BF968C1092F0EC111102BFF1FC116102EFF19C007398DE3585858AC
S11BF98058D7158DDBDB151F98DB10D710398DD220EB8DE797128DE316
S11BF99897139E123910DE213B8DEF8D8220028D88BDF9259F128D8B10
S11BF9B0C10D27F38DD8A782A18427EB863FBDF8EDBDF92520E18DCAF4
S11BF9C8BDF9272003BDF931BDF93BC10D27048DB5A78430019F1220E3
S11BF9E0EC8EFA0ABDF9009E21BDF925BDF925BDF925BDF925BDF923D3
S11BF9F8BDF923BDF923BDF9238E0021BDF9237EF891204343202041B2
S11BFA102020422044502020205820202020592020202055202020508E
S11BFA284320202020530D0A2020202000BDF93BD716108EFA7CA6A0DD
S11BFA401027FE4DAEA1911626F4BDF9271F109E2130864D2A038E008F
S11BFA58219F12D7162605BDF9252003BDF9239E12BDF97BA7800D16A6
S11BFA701026FE1DBDF97BA7847EF891430000410100420200440102B6
S11BFA88470300580402590602550802500A0253FF0200BDF992BDF94C
S11BFAA0272003BDF931BDF92B9F12BDF93BC14427F17EF891BDF9922A
S11BFAB89E12A6844397199E12EC84DD1DEC02DD1FDC1D10931926077F
S11BFAD0DC1F10931B2711BDF8F88E001DBDF92BDC1DDD19DC1FDD1B0E
S11BFAE8F62011C50827D0BDF93B9E12810D1027FD9720093001BDF90D
S11BFB003B810D27B3812D27F381201026FD82BDF97BA78420E60F14A3
S11BFB18BDF93BC15326F9BDF93B34020F10BDF97B80029711BDF992C4
S11BFB3035028139271B813126DEBDF97B0A112704A78020F50C1027DA
S11BFB48CF863FBDF8ED7EF891BDF97B0A1126F10C1026ED8C0000271F
S110FB60029F009E00109E21AF2A7EF891A6
S9030000FC
